S31508006000C8060020F1610008FD610008FF6100086C
S31508006010016200080362000805620008000000002B
S3150800602000000000000000000000000007620008F1
S3150800603009620008000000000B620008856D000870
S315080060400F6200080F6200080F6200080F6200085E
S315080060500F6200080F6200080F6200080F6200084E
S315080060600F6200080F6200080F6200080F6200083E
S315080060700F6200080F6200080F6200080F6200082E
S315080060800F6200080F6200080F6200080F6200081E
S315080060900F6200080F6200080F6200080F6200080E
S315080060A00F6200080F6200080F6200080F620008FE
S315080060B00F6200080F6200080F6200080F620008EE
S315080060C00F6200080F6200080F6200080F620008DE
S315080060D00F6200080F6200080F6200080F620008CE
S315080060E00F6200080F6200080F6200080F620008BE
S315080060F00F6200080F6200080F6200080F620008AE
S315080061000F6200080F6200080F6200080F6200089D
S315080061100F6200080F6200080F6200080F6200088D
S315080061200F6200080F6200080F6200080F6200087D
S315080061300F6200080F6200080F6200080F6200086D
S315080061400F6200080F6200080F6200080F6200085D
S31508006150EE11AA5500F002F800F03AF80AA090E805
S31508006160000C82448344AAF10107DA4501D100F004
S315080061702FF8AFF2090EBAE80F0013F0010F18BF97
S31508006180FB1A43F001031847480E0000680E00008A
S31508006190103A24BF78C878C1FAD8520724BF30C845
S315080061A030C144BF04680C60704700000023002417
S315080061B000250026103A28BF78C1FBD8520728BF09
S315080061C030C148BF0B6070471FB51FBD10B510BD65
S315080061D000F035F81146FFF7F7FF00F0DDFE00F096
S315080061E053F803B4FFF7F2FF03BC00F05BF80000B6
S315080061F00A4885460A4880470A480047FEE7FEE7F8
S31508006200FEE7FEE7FEE7FEE7FEE7FEE7FEE7FEE758
S3150800621005480649064A074B70470000C80600208D
S31508006220956D000855610008C8000020C8060020C2
S31508006230C8020020C802002070477047704775469C
S3150800624000F02CF8AE4605006946534620F00700D4
S31508006250854618B020B5FFF7DBFFBDE820404FF0B4
S3150800626000064FF000074FF000084FF0000B21F032
S315080062700701AC46ACE8C009ACE8C009ACE8C009FF
S31508006280ACE8C0098D46704710B50446AFF30080E8
S315080062902046BDE81040FFF7A4BF0000004870473D
S315080062A06800002001491820ABBEFEE72600020060
S315080062B07047000000BF0748006800F4E060064920
S315080062C00843001D03490860BFF34F8F00BF00BF96
S315080062D0FEE700000CED00E00000FA0500B585B009
S315080062E000210D4800F042FA002812DD6A46002116
S315080062F0094800F04AFA40F267610098884208D1D6
S315080063009DF80B00FF2804D19DF80C0008B9FFF78B
S31508006310D1FF05B000BD00000064004000B58BB099
S315080063200121084600F040FC0121082000F03CFC51
S315080063304FF48070ADF8280048208DF82B000AA984
S31508006340334800F0EBFA4FF40070ADF82800182037
S315080063508DF82B0003208DF82A000AA92C4800F096
S31508006360DDFA01214FF4EA1000F064FB012148062A
S3150800637000F0FAFB274800F0CFF807A800F07DFAEE
S315080063806B4601AA02A94FF4FA7000F087FA0020BA
S315080063908DF822008DF823008DF824008DF825004D
S315080063A08DF826008DF827008DF81E008DF81F0041
S315080063B09DF80400401EC0B28DF820009DF800002C
S315080063C0401EC0B28DF82100BDF80800ADF81C00CB
S315080063D007A9104800F040F900208DF816008DF83E
S315080063E0170001208DF818000020ADF80C00ADF854
S315080063F00E00ADF81000ADF81200ADF8140001203B
S315080064008DF8190003A800F0A3F80BB000BD000032
S31508006410000C01400064004010B500F009F8FFF7D1
S315080064205DFF10BD10B500F039F8FFF777FF10BD16
S3150800643010B51748007850B9164800F09BFD01289A
S3150800644024D1134908700020134908701EE0114A28
S3150800645011490978491C501800F08CFD012815D1FE
S315080064600D480078401C0C4908700A4800780978DD
S3150800647088420BD100200649087006484078FF2854
S3150800648004D10448807808B9FFF714FF10BD00004E
S3150800649015000020240000201400002000B585B057
S315080064A00121480400F060FB0121052000F07CFB77
S315080064B018208DF813000420ADF8100003208DF87D
S315080064C0120004A9124800F029FA04208DF81300D6
S315080064D00820ADF8100004A90D4800F01FFA4FF483
S315080064E0614000900020ADF80400ADF80600ADF854
S315080064F00800ADF80C000C20ADF80A0069460548FE
S3150800650000F0C6FC0121034800F0A8FC05B000BD58
S31508006510000801400044004010B504460B48844278
S3150800652009D10121480600F02FFB00214FF0007029
S3150800653000F02AFB08E00121880600F025FB00216F
S315080065404FF0806000F020FB10BD000000640040A2
S3150800655010B50021837A012202FA03F13D4A126836
S3150800656042F001023B4B1A603A4A1C3212688A43CF
S31508006570384B1C331A60027BCAB9364A0C32126889
S315080065808A43344B0C331A604288C38842EA034371
S31508006590304A4032847A42F834300288838842EAA4
S315080065A003432C4A4032847A02EBC4025360027BCE
S315080065B0012A19D1274A0C3212680A43254B0C3393
S315080065C01A604288038842EA0343224A4032847AA0
S315080065D042F83430C288838842EA03431D4A40326F
S315080065E0847A02EBC4025360C27A3AB9194A121D78
S315080065F012688A43174B1B1D1A6006E0154A121DBE
S3150800660012680A43134B1B1D1A60028932B9114AD4
S31508006610143212688A430F4B14331A600289012A0E
S3150800662006D10C4A143212680A430A4B14331A600C
S31508006630427B012A06D1074A1C3212680A43054BD7
S315080066401C331A60034A126822F00102014B1A60D1
S3150800665010BD00000066004030B502460020002349
S31508006660146824F002041460146844F001041460E9
S3150800667000E05B1C546804F001041CB94FF6FF7473
S31508006680A342F6D1546804F001040CB900206CE06A
S315080066908C79012C04D1146844F08004146003E05A
S315080066A0146824F080041460CC79012C04D1146891
S315080066B044F04004146003E0146824F040041460B5
S315080066C00C7A012C04D1146844F02004146003E009
S315080066D0146824F0200414604C7A012C04D1146840
S315080066E044F01004146003E0146824F010041460E5
S315080066F08C7A012C04D1146844F00804146003E071
S31508006700146824F008041460CC7A012C04D11468A7
S3150800671044F00404146003E0146824F004041460CC
S315080067208C78A407CD7844EA05640D7944EA0544D3
S315080067304D7944EA05540D886D1E2C43D4611468BE
S3150800674024F001041460002300E05B1C546804F084
S3150800675001041CB14FF6FF74A342F6D1546804F045
S3150800676001040CB1002000E0012030BD02460020E3
S3150800677019B9D36803F0030006E0012903D11369A8
S3150800678003F0030000E00020704710B500F5D87349
S3150800679003EB01131B6803F004031372137A53B94E
S315080067A000F5D87303EB01131B6840F2FF7404EA83
S315080067B05353136009E000F5D87303EB01131B6804
S315080067C06FF0604404EAD303536000F5D87303EB13
S315080067D001131B6803F00203537200F5D87303EB29
S315080067E001135B6803F00F03937200F5D87303EB8C
S315080067F001135B681B0AD37400F5D87303EB011306
S315080068009B68D37200F5D87303EB01139B681C0AC7
S31508006810147300F5D87303EB01139B681C0C5473AF
S3150800682000F5D87303EB01139B681B0E937300F5F1
S31508006830D87303EB0113DB68D37300F5D87303EB46
S315080068400113DB681C0A147400F5D87303EB0113F3
S31508006850DB681C0C547400F5D87303EB0113DB6872
S315080068601B0E937421B9C36843F02003C36003E089
S31508006870036943F02003036110BD00218171C171D2
S31508006880017241728172C1728170C17003210171F6
S31508006890022141710121018070470000F0B50546CB
S315080068A00C46002133E01C4810F811001A4E06EB7E
S315080068B0410676783044401C684348F6A04696FB65
S315080068C0F0F700FB176000BB134810F81100124ED2
S315080068D006EB410676783044401C684348F6A046E5
S315080068E096FBF0F02080208800280EDD2088B0F581
S315080068F0806F0ADC084810F811001070064800EB93
S315080069004100407818700120F0BD481CC1B2122918
S31508006910C9D30020F8E70000AC6F00082DE9F04164
S31508006920024600250026002000230024002791F8AF
S3150800693003C00CF00F0591F803C00CF0100CBCF165
S31508006940000F03D091F802C04CEA050591F800C083
S31508006950BCF1000F31D0146800202BE04FF0010C79
S315080069600CFA00F3B1F800C00CEA03069E4220D1E7
S3150800697083004FF00F0C0CFA03F7BC4305FA03FC2F
S315080069804CEA040491F803C0BCF1280F06D14FF075
S31508006990010C0CFA00FCC2F814C00AE091F803C016
S315080069A0BCF1480F05D14FF0010C0CFA00FCC2F8F7
S315080069B010C0401C0828D1D31460B1F800C0BCF13F
S315080069C0FF0F34DD546800202EE000F1080C4FF06C
S315080069D0010808FA0CF3B1F800C00CEA03069E4257
S315080069E021D183004FF00F0C0CFA03F7BC4305FACC
S315080069F003FC4CEA040491F803C0BCF1280F05D146
S31508006A0000F1080C08FA0CF8C2F8148091F803C0D3
S31508006A10BCF1480F07D100F1080C4FF0010808FA3D
S31508006A200CF8C2F81080401C0828CED35460BDE884
S31508006A30F0810000F0B50A46002300240021002555
S31508006A4000F00046B6F1004F02D11D4EF16901E093
S31508006A501B4E7168C0F3034583B200F44016B6F5C1
S31508006A60401F08D121F07061154E766826F07066D1
S31508006A70134F7E6012E000F48016B6F5801F06D12B
S31508006A80032606FA05F4A14341F0706106E0460DB7
S31508006A90360103FA06F6B14341F0706122B1460D9C
S31508006AA0360103FA06F6314300F00046B6F1004F08
S31508006AB002D1034EF16101E0014E7160F0BD0000A4
S31508006AC000000140416170470161704710B500F050
S31508006AD007F800F08FF900F001F810BD62B67047AC
S31508006AE008B50121102000F05FF84FF48050ADF88A
S31508006AF0000003208DF8020010208DF80300694677
S31508006B000448FFF70BFF4FF480510248FFF7DCFFFC
S31508006B1008BD00000010014010B500F065F90446F4
S31508006B200E480068201AB0F5FA7F00D210BD0C484E
S31508006B30007838B901200A49087001030948FFF7A7
S31508006B40C1FF07E00020064908704FF48051054848
S31508006B50FFF7BAFF0148046000BFE7E71C00002002
S31508006B60180000200010014029B1064AD2690243E4
S31508006B70044BDA6104E0034AD2698243014BDA61C5
S31508006B80704700000010024029B1064A1269024304
S31508006B90044B1A6104E0034A12698243014B1A61E5
S31508006BA0704700000010024029B1064A9269024364
S31508006BB0044B9A6104E0034A92698243014B9A6145
S31508006BC0704700000010024030B500210022002462
S31508006BD000232D4D6D6805F00C0121B1042905D05F
S31508006BE0082923D105E0294D056022E0274D0560D7
S31508006BF01FE0254D6D6805F47012234D6D6805F488
S31508006C008034022505EB92421CB9214D5543056097
S31508006C100BE01D4D6D6805F400351DB11C4D55433F
S31508006C20056002E0194D5543056002E0174D056001
S31508006C3000BF00BF144D6D6805F0F0010909154D38
S31508006C406B5C0568DD4045600F4D6D6805F4E061D5
S31508006C50090A104D6B5C4568DD4085600A4D6D6814
S31508006C6005F46051C90A0B4D6B5C4568DD40C5608B
S31508006C70054D6D6805F44041890B074D6B5CC56889
S31508006C80B5FBF3F5056130BD0010024000127A002D
S31508006C9000093D00000000201000002010B500F09B
S31508006CA001F810BD0CB5002001900090334800682B
S31508006CB040F480303149086000BF3048006800F46D
S31508006CC0003000900198401C0190009818B901986E
S31508006CD0B0F5A06FF1D12948006800F4003010B172
S31508006CE00120009001E0002000900098012843D17F
S31508006CF02348006840F010002149086008460068EB
S31508006D0020F0030008600846006840F002000860AA
S31508006D101A48406819494860084640684860084665
S31508006D20406840F4806048600846406820F47C105B
S31508006D3048600846406840F4E8104860084600681D
S31508006D4040F08070086000BF0C48006800F00070D2
S31508006D500028F9D00948406820F003000749486030
S31508006D600846406840F00200486000BF0348406893
S31508006D7000F00C000828F9D10CBD000000100240F4
S31508006D800020024002480068401C0149086070471C
S31508006D902000002010B51148006840F001000F4996
S31508006DA00860084640680E4908400C49486008468D
S31508006DB000680C490840094908600846006820F43C
S31508006DC0802008600846406820F4FE0048604FF4BA
S31508006DD01F008860FFF762FF10BD00000010024028
S31508006DE00000FFF8FFFFF6FE014800687047000044
S31508006DF02000002030B51349B1F1807F00D31DE093
S31508006E0021F07F40401E4FF0E022506150170F22BC
S31508006E10002807DA13071D0E0B4B00F00F04241F7A
S31508006E201D5503E013071C0E084B1C5400BF002019
S31508006E304FF0E02290610720106100BF002000F0AB
S31508006E4007F830BD4019010018ED00E000E400E045
S31508006E5001490860704700002000002021B182899E
S31508006E6042F40052828104E082894DF6FF731A408B
S31508006E708281704702460020B1F5007F00D100BF2D
S31508006E8013880B400BB1012000E00020704700007A
S31508006E902DE9F04786B005460E460024A24600BFF7
S31508006EA0A1460027B08900B100BF2F462C8A4CF6B0
S31508006EB0FF700440F08804432C82AC894EF6F31028
S31508006EC00440B08831890843718908430443AC817A
S31508006ED0AC8A4FF6FF400440B0890443AC8201A84F
S31508006EE0FFF772FE1F48874202D1DDF810A001E0C5
S31508006EF0DDF80CA0A88900F4004040B10AEBCA00EE
S31508006F0000EB0A1031684900B0FBF1F807E00AEB1C
S31508006F10CA0000EB0A1031688900B0FBF1F864205A
S31508006F20B8FBF0F004012009642101FB1089A88947
S31508006F3000F4004040B1322000EBC900B0FBF1F08C
S31508006F4000F00700044308E0322000EB0910642132
S31508006F50B0FBF1F000F00F0004432C8106B0BDE849
S31508006F60F08700000038014001468888C0F3080011
S31508006F707047000010B5044620210648FFF77AFF3F
S31508006F80012805D10348FFF7EFFF2070012010BD47
S31508006F900020FCE700440040FFF798FDFFF742FA9F
S31508006FA003E0FFF7B9FDFFF737FAFAE7050206022D
S31508006FB0060307030803090309040A040B040C045F
S31508006FC00C050D050E050F050F061006100710080F
S31508006FD0F06F0008000000202400000090610008FF
S31508006FE01470000824000020A4060000AC61000804
S31508006FF00000000001020304010203040607080951
S31508007000020406080000000000000000000000005E
S30908007010000000006E
S705080061553C
